:1000000014C024C023C022C021C020C01FC01EC0F5
:100010001DC01CC01BC01AC019C018C017C016C014
:1000200015C014C013C012C011C011241FBECFEDE3
:10003000CDBF10E0A0E6B0E0E4E6F1E002C005903C
:100040000D92A236B107D9F780D08AC0D9CFCF930D
:10005000C2E362D0C150E9F7CF910895CF93C62F84
:10006000843038F4823048F4882371F0813049F0CC
:100070000CC0843051F4939808C04F73833009F456
:10008000405C842F806824D0939A929A929A98B375
:100090009F708C2F807F982B98BB98B39F70892B73
:1000A00088BB9298929838D087B3803F79F4929A1F
:1000B000929A88B3C295C07F8F708C2B88BB88B30F
:1000C0008F70C82BC8BB9298929826D0CF91089574
:1000D00040E0682F84E0C2DF08958FEF87BB8B9AE2
:1000E0008A9A88BB939A929AB2DFB1DFB0DF80E33D
:1000F000EFDFADDF80E3ECDF0FD080E3E9DF88E204
:10010000E7DF87B3807F87BB8CE0E2DF86E0E0DF5C
:1001100082E0DEDF9CDF0895CF93DF931F92CDB79F
:10012000DD2784E4898389819FEF980F9983882351
:1001300041F08981898189819FEF980F998381118D
:10014000F8CF0F90DF91CF9108958FEF87BBC5DF78
:1001500040E060E670E080E081DF8AEA88BBFECFA5
:04016000F894FFCF41
:02016400740025
:00000001FF
